:100000000C9446000C9465000C9465000C946500FB
:100010000C9465000C9465000C9465000C946500CC
:100020000C9465000C9448010C9465000C946500D8
:100030000C9465000C9465000C9465000C946500AC
:100040000C9465000C9465000C9465000C9465009C
:100050000C9465000C9465000C9465000C9465008C
:100060000C9465000C9465000C9465000C9465007C
:100070000C9465000C9465000C9465000C9465006C
:100080000C9465000C9461040C94650011241FBE4F
:10009000CFEFD0E1DEBFCDBF11E0A0E0B1E0EEE9EF
:1000A000FDE000E00BBF02C007900D92A030B10749
:1000B000D9F712E0A0E0B1E001C01D92A732B1076C
:1000C000E1F70E9472010C94CD060C94000080ECC4
:1000D00087B9089583EC86B98091190190911A012E
:1000E0008034910509F070C0809100019091010168
:1000F000A0910201B091030154E0B695A7959795A0
:1001000087955A95D1F790931101809310018091B2
:10011000040190910501A0910601B091070144E00E
:10012000B695A795979587954A95D1F79093130122
:10013000809312018091080190910901A0910A0118
:10014000B0910B0134E0B695A795979587953A95B0
:10015000D1F7909315018093140180910C01909137
:100160000D01A0910E01B0910F0124E0B695A79565
:10017000979587952A95D1F790931701809316014B
:1001800010920001109201011092020110920301DD
:1001900010920401109205011092060110920701BD
:1001A000109208011092090110920A0110920B019D
:1001B00010920C0110920D0110920E0110920F017D
:1001C00010921A01109219013699FECFE091180190
:1001D000F0E0EE0FFF1FEE0FFF1FE050FF4F80819A
:1001E0009181A281B38124B1820F911DA11DB11D06
:1001F00080839183A283B383E0911801F0E0EE0F36
:10020000FF1FEE0FFF1FE050FF4F20813181428121
:10021000538165B1962F80E0AA2797FDA095BA2F4C
:10022000820F931FA41FB51F80839183A283B38382
:10023000809118018F5F809318018091180185309B
:1002400011F41092180180911801882311F480ECA8
:100250000DC080911801813011F481EC07C08091AC
:100260001801823011F482EC01C083EC87B98091CF
:10027000190190911A01019690931A018093190126
:1002800008958BE085BD89EF83BD80E887BF089521
:100290001F920F920FB60F9211248F939F93AF93DB
:1002A000BF9380911B0190911C01A0911D01B09101
:1002B0001E010196A11DB11D80931B0190931C018D
:1002C000A0931D01B0931E01BF91AF919F918F919B
:1002D0000F900FBE0F901F90189585B392E089275D
:1002E00085BB0895EF92FF920F931F93F8940E949D
:1002F0002C040E9441018CE08093260260E070E0B3
:1003000080E090E00E943E040E94670078948FEFA6
:1003100084BB85BB92E3E92EF12C04E110E021E0DF
:1003200030E040E050E060E070E08AE690E00E945B
:100330001B0286E9E82EF12C04EF11E021E030E009
:1003400040E050E060E070E08DE691E00E941B022A
:100350000E941303FDCFEF92FF920F931F93FC01B6
:10036000838994890297F1F482818F3019F0803F5C
:10037000C9F414C087ED91E00E940C0422E3E22E40
:10038000F12C04EF11E021E030E040E050E060E0CB
:1003900070E087ED91E00E941B0204C087ED91E0C0
:1003A0000E940C041F910F91FF90EF900895DF932E
:1003B000CF93CDB7DEB729970FB6F894DEBF0FBE47
:1003C000CDBF80E5898380911001909111019A83BE
:1003D00080911001909111018B8380911201909175
:1003E00013019C8380911201909113018D83809160
:1003F0001401909115019E83809114019091150133
:100400008F83809116019091170198878091160132
:1004100090911701898749E0BE016F5F7F4F81E0AE
:100420000E94720629960FB6F894DEBF0FBECDBFAC
:10043000CF91DF910895CF92DF92EF92FF920F93C9
:100440001F93CF93DF93EC016B01A0E0B0E09A2FF4
:10045000FD0184E0EE0FFF1F8A95E1F7EA0FFB1F15
:10046000E15EFE4F8785882329F09F5F1196AC30AF
:10047000B10569F7692F70E0FB01A4E0EE0FFF1FE3
:10048000AA95E1F7E60FF71FE15EFE4FD183C08327
:10049000D382C2825583448337832683E114F104D7
:1004A00011F4108A08C082E3E816F10411F481E027
:1004B00001C082E0808BFB0134E0EE0FFF1F3A9514
:1004C000E1F7E60FF71FE15EFE4FA089B0E0A5510E
:1004D000BE4F8C91982F9E0D96878F5F8C931187BE
:1004E000008781E08787F89420911B0130911C01DF
:1004F00040911D0150911E01C801A0E0B0E0820FA3
:10050000931FA41FB51FFB0124E0EE0FFF1F2A95C8
:10051000E1F7E60FF71FE15EFE4F82879387A4871E
:10052000B5877894DF91CF911F910F91FF90EF9055
:10053000DF90CF900895CF92DF92EF92FF920F93CA
:100540001F93CF93DF93DC01EB01690120E030E0E2
:10055000622FF90174E0EE0FFF1F7A95E1F7E20FC9
:10056000F31FE15EFE4F8785882331F06F5F2F5FB9
:100570003F4F2C30310561F7262F30E0F90164E060
:10058000EE0FFF1F6A95E1F7E20FF31FE15EFE4FEA
:10059000B183A083D383C28355834483D782C68229
:1005A000E114F10411F4108A08C082E3E816F104A2
:1005B00011F481E001C082E0808BB90194E0660F04
:1005C000771F9A95E1F7620F731F615E7E4FEB0113
:1005D000E889F0E0E551FE4F8081982F9E0D9E87BF
:1005E0008F5F80831987088781E08F8720911B01A7
:1005F00030911C0140911D0150911E01C801A0E0E5
:10060000B0E0820F931FA41FB51FFB018287938761
:10061000A487B587DF91CF911F910F91FF90EF9045
:10062000DF90CF900895EF92FF920F931F93CF9397
:10063000DF93F894E0901B01F0901C0100911D01E4
:1006400010911E0178941092EE018091F1018F5F5C
:100650008093F1018091F101883C49F48091F0018F
:1006600086958093EF011092F0011092F1014FEF07
:100670005FEF20E030E0F901A4E0EE0FFF1FAA9544
:10068000E1F7E20FF31FE15EFE4F8785882399F0C3
:100690008091EE018F5F8093EE0182859385A48522
:1006A000B585E816F9060A071B0728F08685851721
:1006B00010F45685422F2F5F3F4F2C303105D9F66D
:1006C0004F3FB9F18091F0018F5F8093F001842F4B
:1006D000992787FD9095EC01E4E0CC0FDD1FEA95AA
:1006E000E1F7C80FD91FC15EDE4FE881F9816C8147
:1006F0007D818A819B8109958E819F81892B49F417
:100700001F86E889F0E0E551FE4F808181508083AB
:1007100010C02A853B854C855D8588859985A0E03C
:10072000B0E0820F931FA41FB51F8A879B87AC87F9
:10073000BD8781E0DF91CF911F910F91FF90EF90E6
:1007400008959C01DB0160E070E0FB0144E0EE0FE6
:10075000FF1F4A95E1F7E60FF71FE15EFE4F80812C
:1007600091818217930719F58785882301F1F89401
:1007700020911B0130911C0140911D0150911E01DF
:10078000CD01A0E0B0E0820F931FA41FB51FFB01B5
:1007900024E0EE0FFF1F2A95E1F7E60FF71FE15E59
:1007A000FE4F82879387A487B587789408956F5FFB
:1007B0007F4F6C30710549F60895AC0120E030E0C0
:1007C000F901A4E0EE0FFF1FAA95E1F7E20FF31F76
:1007D000E15EFE4F8081918184179507B9F487858A
:1007E0008823A1F020911B0130911C0140911D0133
:1007F00050911E01CB01A0E0B0E0820F931FA41F17
:10080000B51F82879387A487B58708952F5F3F4FD1
:100810002C303105A9F60895AC0120E030E0F90153
:10082000B4E0EE0FFF1FBA95E1F7E20FF31FE15EB0
:10083000FE4F808191818417950741F41786E089E6
:10084000F0E0E551FE4F8081815080832F5F3F4F64
:100850002C30310521F7089580E090E0FC0124E080
:10086000EE0FFF1F2A95E1F7E80FF91FE15EFE4F3B
:10087000178601968C30910589F70895809126029C
:10088000880F81608093720080E480937000E1E7BC
:10089000F0E080818C7F80832FEF2093730085ECC4
:1008A0008093740081E090E09093F5018093F401CF
:1008B0001092F3012093200210920A021092090272
:1008C00008951F920F920FB60F920BB60F9211243C
:1008D000EF92FF920F931F932F933F934F935F934A
:1008E0006F937F938F939F93AF93BF93EF93FF93F8
:1008F0008091F4019091F501817C09F4CBC0809145
:10090000710090E0887F90708038910561F18138A6
:100910009105ACF48836910509F48AC089369105B1
:100920002CF48036910509F0B3C09AC08037910548
:1009300009F496C08837910509F0AAC079C08039BA
:10094000910589F0813991052CF48838910509F0D9
:100950009FC096C08839910509F492C0803A9105EC
:1009600009F096C093C08091F4019091F501803414
:10097000910581F4809173008093F7018FEF80934C
:10098000200280E890E09093F5018093F4011092AA
:10099000F3017CC08091F4019091F50180389105BC
:1009A00009F074C09091F3018091F7019817A0F4B9
:1009B0008091F301E82FF0E090917300EA50FE4F30
:1009C00092838F5F8093F301909120028091730056
:1009D0008927809320025AC08091F301803111F55C
:1009E0008091730080930802909120028091080208
:1009F000981719F081E090E002C082E090E09093B7
:100A00000A0280930902EE24FF2400E010E020E0B7
:100A100030E040E050E066EF71E08BEA91E00E9448
:100A20009B022EC08091F3018F5F8093F3012EC053
:100A3000809124028F5F80932402809121028A306A
:100A400078F422E3E22EF12C02E310E020E030E023
:100A500040E050E060E070E086E396E00E949B0298
:100A6000809173008093F60110920A02109209029D
:100A70001092F30185EC8093740080E490E07DC0D7
:100A800081E090E09093F5018093F40185ECD5C06E
:100A900085E4D3C08091710090E0887F90708032AF
:100AA000910509F49CC08132910554F4803191057F
:100AB00099F088319105D1F0089709F0B7C00CC0C2
:100AC0008033910509F45EC08833910509F460C054
:100AD000889709F0ABC011C080910B02809373001E
:100AE00085E88093740088E090E047C01092F2019E
:100AF00080910C02809373003BC08091F2018131A0
:100B0000D9F485E98093740080E290E09093F50138
:100B10008093F4011092210280912202909123028D
:100B20000196909323028093220260E070E08EE3AE
:100B300094E00E94DD0383C09091F20180910C0249
:100B4000981750F080911D02809373008091F201FC
:100B50008F5F8093F2010CC09091F201E92FF0E0D9
:100B6000E55FFD4F8281809373009F5F9093F20158
:100B700085E88093740080E190E09093F501809384
:100B8000F4015DC0809124028F5F809324022CC009
:100B9000809124028F5F8093240260E070E08EE3F6
:100BA00094E00E94DD03809121028A3080F492E378
:100BB000E92EF12C02E310E020E030E040E050E0CC
:100BC00060E070E086E396E00E949B0206C088E247
:100BD00090E09093F5018093F40185E82EC0809118
:100BE00025028F5F8093250260E070E08EE394E041
:100BF0000E94DD03809121028A3080F482E3E82E96
:100C0000F12C02E310E020E030E040E050E060E052
:100C100070E086E396E00E949B0206C088E290E0C6
:100C20009093F5018093F40185E907C084E090E09A
:100C30009093F5018093F40185E080937400FF9117
:100C4000EF91BF91AF919F918F917F916F915F9144
:100C50004F913F912F911F910F91FF90EF900F9027
:100C60000BBE0F900FBE0F901F901895EF92FF9242
:100C70000F931F938091F4019091F501019771F00A
:100C800042E3E42EF12C05E010E020E030E040E00B
:100C900050E060E070E086E396E01DC01092F20143
:100CA00085EA8093740082E090E09093F501809350
:100CB000F401809121028F5F8093210232E3E32EC1
:100CC000F12C00E117E220E030E040E050E060E08D
:100CD00070E08EE394E00E941B021F910F91FF9041
:100CE000EF900895EF92FF920F931F93582F8091EA
:100CF0002102882309F448C0809121028A3009F436
:100D000043C081E03CC08FEF80931D02DB0120E0F7
:100D100030E00DC08C91F901E55FFD4F8283809139
:100D20001D029D91892780931D022F5F3F4F24173D
:100D300088F381E080932102852F90E0880F991F2E
:100D400080930B0240930C021092F20185EA80938B
:100D5000740082E090E09093F5018093F40152E3F7
:100D6000E52EF12C05E010E020E030E040E050E01E
:100D700060E070E08EE394E00E941B0280E01F912F
:100D80000F91FF90EF9008958091F4019091F501FB
:0E0D9000019709F4B8CF82E0F2CFF894FFCFBC
:00000001FF
